:020000000140BD
:020003000157A3
:05000B0002005101405C
:2000400075811CD2AFD2A9D28C12005A12001B80FB438CDC050832050832740075F000F529
:200060000985F00A740075F000F51785F018748075F025C0E0C0F0120C3C15811581120C14
:200080008B796C7A0EE98AF0C0E0C0F0120C5F158115811201F312018B1202061208D11251
:2000A000025612037C12048812064E1205F21206FD1208F11209DE020096227F09120D1AB6
:2000C000740078FC120D0EF6740075F00008F608A6F078FC120D0EE6120D407B0A120D37DF
:2000E000120E0D45F0700302013D801678FD120D0EE60886F0120DCA18F608A6F0120DD3C8
:2001000080D0741175F000C0E0C0F0120C7315811581120C8BC0E0C0F0120C9B15811581BA
:2001200078FC120D0EF608E60886F079F6120D13120D3078FC120D0EE6F70200EC78FD12D9
:200140000D0EE60886F079F6120D13120D307400F778FD120D0EE60886F07B007C00120EA8
:200160000445F0700302017074FF75F0FF02018679F6120D13E98AF0C0E0C0F0120CBB15BE
:200180008115810201867FF7020D29E598540175F0007B007C00120E0D45F070030201B358
:2001A000120C8BC0E0C0F0120C9B15811581F5120201B774FFF51222E598540175F0007B52
:2001C000007C00120E0D45F070030201D5120CB0F5120201D974FFF51222120243799F7AC0
:2001E0000EE98AF0C0E0C0F0120C5F158115811201F322799B7A0EE98AF0C0E0C0F0120C00
:200200005F1581158122E512120D407B0A120D37120E0445F0700302022F796C7A0EE98A21
:20022000F0C0E0C0F0120C5F158115811201F322C292746475F000C0E0C0F0120CF1158127
:20024000158122D292746475F000C0E0C0F0120CF11581158122E512120D407B65120D370C
:20026000120E0445F07003020353120230D2B3D2B4C2B5D2B2C2B6C2B7120A55C2B3746461
:2002800075F000C0E0C0F0120CF115811581E50E75F0007B557C00120E0445F070030203F9
:2002A0001AC295746475F000C0E0C0F0120CF115811581C2A700D2A7749675F000C0E0C054
:2002C000F0120CF115811581D292746475F000C0E0C0F0120CF115811581C292746475F036
:2002E00000C0E0C0F0120CF115811581C2A700D2A7749675F000C0E0C0F0120CF115811518
:2003000081D292746475F000C0E0C0F0120CF115811581C292D29502032EC2A7740A75F0F6
:2003200000C0E0C0F0120CF115811581D2A7740A75F000C0E0C0F0120CF115811581D2B3C6
:20034000746475F000C0E0C0F0120CF1158115811201DA22851380C2970000000000D297EC
:2003600000000000C29700000000E5144480F5A0C2B574FFF580E58075F00022E512120D71
:20038000407B77120D37120E0445F07003020487120230D295C297D2B3C2B4D2B5D2B2D2A0
:2003A000B6D2B7D2A7120A55C2B3746475F000C0E0C0F0120CF115811581740075F000F509
:2003C0001585F016740075F000F50985F00AE509850AF0AB17AC18120E1745F0700302044F
:2003E000728012E509850AF0120DCAF50985F00A120DD380D9741175F000C0E0C0F0120C83
:200400007315811581E509850AF0F51385F014851380D29700000000C29700000000E5146C
:200420004480F5A0120A55120CB0F580741375F000C0E0C0F0120C7315811581E515851621
:20044000F02580C5F03400C5F0F51585F016120A2AE50E75F0007B557C00120E0445F07021
:200460000302046A3096FD02046FD2A630A6FD0203E3D2B3746475F000C0E0C0F0120CF17D
:20048000158115811201DA2205810581E512120D407B72120D37120E0445F0700302054069
:2004A000740075F000F51585F016120230D295C297D2B3D2A7C2B4D2B5C2B2D2B6D2B774D6
:2004C00031F50D740075F00078FD120D0EF608A6F078FD120D0EE60886F0AB17AC18120E2E
:2004E0001745F0700302053D801678FD120D0EE60886F0120DCA18F608A6F0120DD380D185
:2005000078FD120D0EE60886F0F51385F014120354F50CE5158516F0250CC5F03400C5F086
:20052000F51585F016E50C75F000C0E0C0F012054515811581D2B512056C0204EA1201DA11
:20054000158115812278FB120D0EE6F50BE50B75F0007B047C00120DB9F50B12058F78FB86
:20056000120D0EE6540FF50B12058F221201B87B137C00120E0445F0700302058E1201B83C
:200580007B117C00120E0D45F0600302057D22E50B75F0007B097C00120E2745F0700302A2
:2005A00005B7E50B243775F000C0E0C0F0120C73158115810205C9E50B243075F000C0E0A9
:2005C000C0F0120C731581158122E58075F0007BFF7C00120E0D45F070030205F17430F566
:2005E0000DE51B851CF0120DCAF51B85F01C120DD322E512120D407B62120D37120E0445CD
:20060000F0700302064D120230D2B4D2B5C2B2D2B6C2B774FFF580E580F50CE50C541CF5B8
:200620000C74A475F00EC0E0C0F0E50C75F0007B027C00120DB9C0E0C0F0740275F000126F
:200640000AE715811581158115811201DA22E512120D407B6C120D37120E0445F0700302E1
:2006600006FC120230C2B3E50E75F0007B557C00120E0445F0700302067CC295D2A7D2B475
:20068000D2B5D2B2D2B6D2B7746475F000C0E0C0F0120CF115811581120A4D740575F0002F
:2006A000C0E0C0F0120CF115811581C2B6C2B7120A55120A4D740575F000C0E0C0F0120C98
:2006C000F115811581C2B5D2B6C2B7120A55120A4D740575F000C0E0C0F0120CF1158115C3
:2006E00081D292746475F000C0E0C0F0120CF115811581C292D295D2B51201DA22E51212F3
:200700000D407B63120D37120E0445F0700302074174BC75F00EC0E0C0F0E5158516F012B8
:200720000DDD2401C5F03400C5F0C0E0C0F0740275F000120AE71581158115811581120173
:20074000DA22120230C297D295D2B3D2A7C2B4D2B5C2B2C2B6C2B7743175F000F51385F0B2
:2007600014120354F510120A55740075F001F51385F014120354F511E51075F0007B517C0A
:2007800000120E0445F0700CE51075F0007B527C00120E0445F070030207A2E510F50E0270
:2007A00007C0E51175F0007B557C00120E0445F070030207BCE511F50E0207C074FFF50E02
:2007C00074FFF50FD2B522120742E50E75F000900830020D49740075F010F51985F01A029E
:2007E0000850740075F010F51985F01A020850740075F020F51985F01A020850740075F0F8
:2008000020F51985F01A020850740075F050F51985F01A020850740075F050F51985F01ADB
:20082000020850740075F000F51985F01A0208502308FF001608650009085500FC07620016
:20084000EF075200E2076100D507510000005008740075F000F51585F016740075F000F545
:200860001B85F01CD2B3D2A7C2B4D2B5C2B2D2B6D2B77431F50D740075F000F50985F00A4F
:20088000E509850AF0AB19AC1A120E1745F070030208D08012E509850AF0120DCAF509853D
:2008A000F00A120DD380D9E509850AF0F51385F014120354F50CE5158516F0250CC5F034EC
:2008C00000C5F0F51585F0161205CAD2B502089522E512120D407B73120D37120E0445F0B2
:2008E00070030208F01200BBF51785F0181201DA22E512120D407B67120D37120E0445F02F
:2009000070030209DD1207C7E50E75F0007BFF7C00120E0D45F070030209CA74CC75F00EF1
:20092000C0E0C0F0E50E75F000C0E0C0F0740275F000120AE71581158115811581E50F7520
:20094000F0007BFF7C00120E0445F0700302096074DB75F00EC0E0C0F0120C5F15811581BF
:20096000E50F75F0007B057C00120E0445F0700302098374E075F00EC0E0C0F0120C5F151F
:2009800081158174E475F00EC0E0C0F0E51B851CF0C0E0C0F0740275F000120AE7158115BB
:2009A000811581158174F875F00EC0E0C0F0E5178518F0C0E0C0F0740275F000120AE7158F
:2009C000811581158115810209DA740B75F00FC0E0C0F0120C5F158115811201DA22E512FD
:2009E000120D407B70120D37120E0445F07003020A291207C7741D75F00FC0E0C0F0E50E2E
:200A000075F000C0E0C0F0E51B851CF0C0E0C0F0E5178518F0C0E0C0F0740475F000120A6E
:200A2000E77FF8120D1A1201DA22E50E75F0007B557C00120E0445F07003020A45C2A700E6
:200A4000D2A7020A4CC2A7000000D2A722C2A7120A9ED2A72205810581740075F00078FDA9
:200A6000120D0EF608A6F078FD120D0EE60886F07B017C00120DE445F07003020A998016D1
:200A800078FD120D0EE60886F0120DCA18F608A6F0120DD380D1020A801581158122058118
:200AA0000581740075F00078FD120D0EF608A6F078FD120D0EE60886F07B147C00120DE48D
:200AC00045F07003020AE2801678FD120D0EE60886F0120DCA18F608A6F0120DD380D1020A
:200AE0000AC9158115812223F42581F8868208868308E4FEFF93700122B42555A3E493B4FC
:200B00002D06430780A3E493B4300343074024D0B40A00500CCE75F00AA42EFEA3E4938098
:200B2000EDE493B46413E60886F030F708430720120DDAA6F018F68003B4750543070A8007
:200B40001CB478054307108014B46F0B430708800C120C79A3809BB462624307027A00C0FB
:200B600004C005C006C007AB0753031F7C00E60886F0120D86A6F018F6EDD007D006D00560
:200B8000D0042430B43A0040022407C0E00AE645F070CCA902EF30E506742D120C790A12C8
:200BA0000C1DD0E0120C79D9F90808EF30E7A5EAC39E50A07420120C790A80F3B4630BAA89
:200BC00001120C1DE6120C7980DFB4732BC082C08386820886837A00E4936004A30A80F893
:200BE0008683188682120C1DE493A36005120C7980F6D083D08280B1B4691986017A00E711
:200C00006004090A80F9120C1D8601E7609B120C790980F7F97A01120C1DE980A8EE601B00
:200C20008FF020F716C002EAC39E500D742030F6027430120C790A80EED0022278FB120DA9
:200C40000E8603088604748075F070120D86120DDA758921F58DF58B758859759852227894
:200C6000FB120D0E8682088683E493602D120C79A380F678FB120D0EE63099FDC299F5994A
:200C8000B40A17740D80F2E430980C3098FDC298E599B40D02740A75F0002278FB120D0ECF
:200CA000E63099FDC299F5992274FFF5F030980A3098FDC298E59975F0002278FB120D0E8F
:200CC0008601E4FBFCFFE709B42D030FE709C39430B40A005012FA740A75F000120D722AA1
:200CE000FBE5F03400FC80E4EB8CF0DF03020DDA2278FB120D0E8603088604BB0004BC0006
:200D0000012279E5A3D9FD1BBBFFF01C80F4C82581C822C92581C97A0022D083D082CF25BF
:200D200081F581CFC082C08322CF2581F581CF2229F9E5F03AFA227C00CB30E7011CCB22B5
:200D400075F00030E70215F022FDE493A3FEE493A3FF4E7009E493FE740193FF800BE4937B
:200D6000A3B5050BE493B5F0068F838E82E473A380D8FEEBA4FD8EF0ECA4FCEB8EF0A4C50F
:200D8000F02C2DC5F022C002C001AAF0F97E007D007F11C3E933F9EA33FADF08F5F0E9D01E
:200DA00001D00222ED33FDEE33FEC3ED9BF5F0EE9C40E0ADF0FED380DBBB000122C3C5F009
:200DC00013C5F013DBF722120DCA04700205F022120DD314B4FF0215F022120DD3F4C5F051
:200DE000F4C5F022120E374029801E120E3740227017801E120E3740107017800C120E37DB
:200E000050108005120E4B6009E4F5F022120E4B60F7E4F5F00422120E4B40F680EB120E51
:200E20004B40EF70E480EB120E4B40DD70E480D9120E4B50DD80D2C39BC5F09C20E707207D
:200E4000D207C345F02220D2F9D322C5F0C39C7003E5F09B22FBE493CB22FCE493FB740164
:200E600093CC22FAE493F9740193CA220A20456173792D446F776E6C6F61646572205633F2
:200E80002E3020666F722041544D454C2038394335312F35322F35355744000A203E000A84
:200EA000206F6B000A206C6F636B2062697420312C322C33203D2025303362000A204348DC
:200EC0004B53554D203D2025303478000A20666F756E6420383943253278002D3132560085
:200EE0002D3556000A206E6F6E626C616E6B202575206279746573000A206279746573204B
:200F0000636F756E746572202575000A204E6F7420666F756E642038394378780025782CF3
:060F200025752C2575006B
:00000001FF
